:020000040000FA
:100000001AEF1EF012000100B83C000000010000D1
:10001000B2000000D9CFE6FFE1CFD9FFFF0EE76EB7
:10002000FD0EDBCF00F0FE0EDBCF01F0E750001637
:10003000016A0050A96EFD0EDBCF00F0FE0EDBCF93
:1000400001F001C000F0016A030E0014AA6EA69E22
:10005000A69CA680A85000D0E552E7CFD9FF120099
:10006000D9CFE6FFE1CFD9FF020EE126DE6ADD6AD5
:10007000FD0EDBCF00F0FE0EDBCF01F001C000F083
:10008000016A030E0014AA6EFF0EE76EFD0EDBCFB1
:1000900000F0FE0EDBCF01F0E7500016016A0050C1
:1000A000A96EFC0EDB50A86EA69EA684A69CF2AE9E
:1000B00004D0F29E010EDE6EDD6A550EA76EAA0E0A
:1000C000A76EA682A1A8FED7A198A694D9CFE9FFD2
:1000D000DACFEAFF010EEE1801E1ED5001E1F28EF8
:1000E000020EE15C02E2E16AE552E16EE552E7CF21
:1000F000D9FF1200D9CFE6FFE1CFD9FFE652D950A0
:10010000FD0FE96EFF0EDA20EA6EFF0ED880EE5486
:10011000030EED5401E21BD0FD0EDBCFE6FFFE0E19
:10012000DBCFE6FF77DFE552E552DF6EDF5001E11E
:100130000ED0DFCFE6FFE66A4AEC0AF0E552E55260
:10014000FD0EDB2AFE0E01E3DB2ADF50D8E1E80ECC
:10015000E66E030EE66EE66AE66A67EC0AF0E552C2
:10016000E552E552E552E552E552E7CFD9FF1200DC
:10017000D9CFE6FFE1CFD9FF030EE126010EDB6AFE
:10018000020EF36EF3CFDBFFFD0EDBCF00F0FE0EB1
:10019000DBCF01F0013404E200500008000E0154EE
:1001A00018E2140EE76E010EDBCF00F0020EDBCF7B
:1001B00001F0E7500026000E0122010E00C0DBFF17
:1001C000020E01C0DBFFFD0EDB06FE0E01E2DB06C8
:1001D000DBD70101B26BB36B140EB25D000EB359E5
:1001E0001CE2010EDB50B2250001006E020EDB5056
:1001F0000101B3210001016E00C0E6FF01C0E6FF6E
:1002000009DFE552E552DF6EDFCFE6FFC6D8E552E3
:100210000101B22B000EB323DFD7030EE15C02E233
:10022000E16AE552E16EE552E7CFD9FF1200D9CF7E
:10023000E6FFE1CFD9FF040EE126200EDE6EA10E0F
:10024000DE6E070EDE6EDD6ADD52DD52D9CFE9FFCC
:10025000DACFEAFFD880000EEE54000EEE54000E06
:10026000EE54000EEE540AE2D9CFE9FFDACFEAFFEE
:10027000EE06000EEE5AEE5AEE5AE8D7040EE15C96
:1002800002E2E16AE552E16EE552E7CFD9FF1200E2
:10029000D9CFE6FFE1CFD9FF020EE126C580C5B078
:1002A000FED7FE0EDBCFE6FF6EEC1CF0E552DF6EF4
:1002B000FF0EDF5C04E1010EC9CFDBFFC69EFD0E21
:1002C000DBCFE6FF6EEC1CF0E552DF6EC584C5B4F3
:1002D000FED7DF50006E020EE15C03E200D0E16A5F
:1002E000E552E16E0050E552E7CFD9FF1200D9CFB9
:1002F000E6FFE1CFD9FFE6520101DC6BFE0EDB50D9
:10030000F00B0809DF6E040EDF10E66EDAC1E6FFBF
:10031000BFDFE552E5520101DC6F010EE66E36ECFF
:100320001EF0E552FB0EDF14E66EDAC1E6FFB0DF29
:10033000E552E5520101DC6F010EE66E36EC1EF06F
:10034000E552FD0EDB5024E0FE0EDB38F00BF00B27
:100350000809DF6E040EDF10E66EDAC1E6FF98DFF3
:10036000E552E5520101DC6F020EE66E36EC1EF03E
:10037000E552FB0EDF14E66EDAC1E6FF89DFE552D7
:10038000E5520101DC6F010EE66E36EC1EF0E5521F
:10039000E552E552E7CFD9FF1200D9CFE6FFE1CF12
:1003A000D9FFE652FE0EDB50F00B08090109DF6EA3
:1003B000040EDF10E66EDAC1E6FF6ADFE552E552B1
:1003C0000101DC6F020EE66E36EC1EF0E552FB0E0C
:1003D000DF14E66EDAC1E6FF5BDFE552E5520101AC
:1003E000DC6F010EE66E36EC1EF0E552FE0EDB38D9
:1003F000F00BF00B08090109DF6E040EDF10E66E4A
:10040000DAC1E6FF45DFE552E5520101DC6F010E7E
:10041000E66E36EC1EF0E552FB0EDF14E66EDAC136
:10042000E6FF36DFE552E5520101DC6F010EE66EB4
:1004300036EC1EF0E552E552E552E7CFD9FF120047
:10044000F40EE66ECAEC1DF0E552E66A300EE66E7A
:100450004EDFE552E552640EE66ECAEC1DF0E55241
:10046000E66A300EE66E43DFE552E5520A0EE66EAE
:10047000CAEC1DF0E552E66A300EE66E38DFE55252
:10048000E552050EE66ECAEC1DF0E552E66A200E56
:10049000E66E2DDFE552E552050EE66ECAEC1DF064
:1004A000E552010EE66E280EE66E21DFE552E552BA
:1004B000050EE66ECAEC1DF0E552010EE66E080E62
:1004C000E66E15DFE552E552050EE66ECAEC1DF04C
:1004D000E552010EE66EE66E0ADFE552E552050EC4
:1004E000E66ECAEC1DF0E552010EE66E060EE66EF3
:1004F000FEDEE552E552050EE66ECAEC1DF0E55251
:10050000010EE66E0C0EE66EF2DEE552E552140EBA
:10051000E66ECAEC1DF0E5521200D9CFE6FFE1CF3E
:10052000D9FF020EE126DE6ADD6AFD0EDBCFF6FFA3
:10053000FE0EDBCFF7FF0800F55021E0DECF00F024
:10054000DDCF01F0D890015004E6140E005C000EDF
:10055000015815E2FD0EDBCFF6FFFE0EDBCFF7FFF5
:100560000800F550E66E19DFE552FD0EDB2AFE0E9F
:1005700001E3DB2ADF2A010E01E3DB2AD6D7020ED4
:10058000E15C02E2E16AE552E16EE552E7CFD9FFB4
:100590001200D9CFE6FFE1CFD9FF020EE126DE6AD5
:1005A000DD6AFD0EDBCFE9FFFE0EDBCFEAFFEF5089
:1005B00020E0DECF00F0DDCF01F0D890015004E65E
:1005C000140E005C000E015814E2FD0EDBCFE9FFB3
:1005D000FE0EDBCFEAFFEF50E66EDFDEE552FD0EEA
:1005E000DB2AFE0E01E3DB2ADF2A010E01E3DB2A10
:1005F000D8D7020EE15C02E2E16AE552E16EE55213
:10060000E7CFD9FF1200D9CFE6FFE1CFD9FF020E25
:10061000E126FD0EDBCF1EF0FE0EDBCF1FF0040E39
:100620001E1801E11F5031E0030E1E1801E11F509A
:1006300021E0020E1E1801E11F5011E0010E1E18EC
:1006400001E11F5001E02CD0800EDE6EDD6A010E4C
:10065000E66E800EE66E4BDEE552E55221D0C00E0E
:10066000DE6EDD6A010EE66EC00EE66E40DEE5521D
:10067000E55216D0940EDE6EDD6A010EE66E940E23
:10068000E66E35DEE552E5520BD0D40EDE6EDD6A45
:10069000010EE66ED40EE66E2ADEE552E55200D07B
:1006A000020EE66ECAEC1DF0E552000EE66EE66A3A
:1006B0005FDDE552E552020EE66ECAEC1DF0E55232
:1006C000010EE66EDFCFE6FF12DEE552E552020EC6
:1006D000E15C02E2E16AE552E16EE552E7CFD9FF63
:1006E000120037D8C580C5B0FED7120032D8C582F7
:1006F000C5B2FED712002DD8C584C5B4FED71200EE
:10070000D9CFE6FFE1CFD9FF9E96FE0EDB50C96E32
:100710009EA6FED7E552E7CFD9FF1200D9CFE6FF5C
:10072000E1CFD9FF16D8C586C5B6FED7C7A0FED77C
:10073000FE0EDBCFE6FF19D8E552C95000D0E552D6
:10074000E7CFD9FF1200280EC66E180EC86E9E960F
:100750001200640EE66EE66AE66AE66A67EC0AF084
:10076000E552E552E552E5521200D9CFE6FFE1CF5E
:10077000D9FFFE0EDB5002E0C58A01D0C59AC588BC
:10078000C5B8FED7E552E7CFD9FF1200D9CFE6FFB3
:10079000E1CFD9FF0E0EE126F90EDBCFDEFFDBCF76
:1007A000DDFFF80EDBCF02F0000EE76E0218E8AEB8
:1007B00002D0023403D0E750D880025402E3070E7F
:1007C00012D0F80EDBCF03F0160EE76E0318E8AE7A
:1007D00002D0033403D0E750D880035402E2170E4E
:1007E00002D0F80EDB28006E016A00BE0168080E18
:1007F00000C0DBFF090E01C0DBFF020EDB6A030E47
:10080000DB6AFB0EDBCF00F0FC0EDBCF01F0FD0E50
:10081000DBCF02F0FE0EDBCF03F0226A236A246AEC
:10082000256A00C01DF001C01EF002C01FF003C009
:1008300020F0E5EC17F0010A33E1F90EDBCFE9FF18
:10084000DB2AFA0EDBCFEAFF01E3DB2A2D0EEF6E87
:10085000FB0EDBCF00F0FC0EDBCF01F0FD0EDBCF9B
:1008600002F0FE0EDBCF03F0226A236A800E246EB4
:10087000BF0E256E00C01DF001C01EF002C01FF0AB
:1008800003C020F009EC17F0FB0E1DC0DBFFFC0ECF
:100890001EC0DBFFFD0E1FC0DBFFFE0E20C0DBFF16
:1008A000FB0EDBCF00F0FC0EDBCF01F0FD0EDBCF4B
:1008B00002F0FE0EDBCF03F0226A236A246A256A67
:1008C00000C01DF001C01EF002C01FF003C020F0E8
:1008D000DCEC17F0010A4AE1FB0EDBCF00F0FC0E66
:1008E000DBCF01F0FD0EDBCF02F0FE0EDBCF03F01D
:1008F000226A236A800E246E3F0E256E00C01DF012
:1009000001C01EF002C01FF003C020F0E5EC17F09C
:10091000010A2CE1006A016A200E026E410E036E8C
:10092000D950FB0FE96EFF0EDA20EA6EEECF1DF014
:10093000EECF1EF0EECF1FF0EFCF20F000C022F080
:1009400001C023F002C024F003C025F009EC17F029
:1009500020C0EDFF1FC0EDFF1EC0EDFF1DC0EFFF6B
:10096000020EDB06030E01E2DB06B6D7FB0EDBCF81
:1009700000F0FC0EDBCF01F0FD0EDBCF02F0FE0E2F
:10098000DBCF03F0226A236A200E246E410E256E0F
:1009900000C01DF001C01EF002C01FF003C020F017
:1009A000E5EC17F0010A2EE0FB0EDBCF00F0FC0EA9
:1009B000DBCF01F0FD0EDBCF02F0FE0EDBCF03F04C
:1009C000226A236A200E246E410E256E00C01DF09F
:1009D00001C01EF002C01FF003C020F0B6EC16F0FC
:1009E000FB0E1DC0DBFFFC0E1EC0DBFFFD0E1FC09B
:1009F000DBFFFE0E20C0DBFF020EDB2A030E01E34D
:100A0000DB2AB4D7020EDBCF00F0030EDBCF01F000
:100A1000D950080FE96EDACFEAFF0050EE260150F8
:100A2000ED22010EF36E040EF3CFDBFF050EDB6A41
:100A3000040EDBCF1EF0050EDBCF1FF0F1EC15F03E
:100A40000A0E1DC0DBFF0B0E1EC0DBFF0C0E1FC00D
:100A5000DBFF0D0E20C0DBFF040EDBCF00F0050E28
:100A6000DBCF01F0080EDBCF02F0090EDBCF03F085
:100A700001500318E8AE02D0033404D00250005CE9
:100A8000035001582EE20A0EDBCF00F00B0EDBCF35
:100A900001F00C0EDBCF02F00D0EDBCF03F0226A6B
:100AA000236A200E246E410E256E00C01DF001C089
:100AB0001EF002C01FF003C020F0B6EC16F00A0EC4
:100AC0001DC0DBFF0B0E1EC0DBFF0C0E1FC0DBFFCB
:100AD0000D0E20C0DBFF040EDB2A050E01E3DB2A2E
:100AE000BBD70A0EDBCF04F00B0EDBCF05F00C0EEC
:100AF000DBCF06F00D0EDBCF07F0226A236A246AF3
:100B0000400E256E04C01DF005C01EF006C01FF08B
:100B100007C020F0B6EC16F01DC000F01EC001F0BA
:100B20001FC002F020C003F0D950FB0FE96EFF0E8A
:100B3000DA20EA6EEECF1DF0EECF1EF0EECF1FF002
:100B4000EFCF20F000C022F001C023F002C024F05B
:100B500003C025F020EC16F020C0EDFF1FC0EDFF14
:100B60001EC0EDFF1DC0EFFFFB0EDBCF00F0FC0E43
:100B7000DBCF01F0FD0EDBCF02F0FE0EDBCF03F08A
:100B8000226A236A200E246E410E256E00C01DF0DD
:100B900001C01EF002C01FF003C020F0E5EC17F00A
:100BA000010A13E0FB0EDB6AFC0EDB6A800EF36EBB
:100BB000FD0EF3CFDBFF3F0EF36EFE0EF3CFDBFF38
:100BC000020EDB2A030E01E3DB2A020EDBCF00F06C
:100BD000030EDBCF01F00001800E01145FE0F90E7F
:100BE000DBCFE9FFDB2AFA0EDBCFEAFF01E3DB2AEA
:100BF000300EEF6EF90EDBCFE9FFDB2AFA0EDBCF0A
:100C0000EAFF01E3DB2A2E0EEF6E080EDBCF00F0C9
:100C1000090EDBCF01F0800E011414E0020EDBCFD1
:100C200002F0030EDBCF03F0080EDB50025C006E17
:100C3000090EDB500358016E020E00C0DBFF030EED
:100C400001C0DBFF040EDB68050EDB68040EDBCFA2
:100C500000F0050EDBCF01F0020EDBCF02F0030E39
:100C6000DBCF03F003500118E8AE02D0013404D00A
:100C70000050025C0150035811E2F90EDBCFE9FF8E
:100C8000DB2AFA0EDBCFEAFF01E3DB2A300EEF6E40
:100C9000040EDB06050E01E2DB06D8D7040EDB6A84
:100CA000050EDB6A040EDBCF00F0050EDBCF01F092
:100CB000080EDBCF02F0090EDBCF03F00150031862
:100CC000E8AE02D0033404D00250005C0350015857
:100CD00001E3ACD0FB0EDBCF1DF0FC0EDBCF1EF032
:100CE000FD0EDBCF1FF0FE0EDBCF20F076EC17F011
:100CF000060E1EC0DBFF070E1FC0DBFF300EE76EC7
:100D0000060EDBCF00F0070EDBCF01F0E750002628
:100D1000000E0122F90EDBCFE9FFDB2AFA0EDBCF52
:100D2000EAFF01E3DB2A00C0EFFF040EDBCF00F097
:100D3000050EDBCF01F0020EDB50001803E1030EBD
:100D4000DB5001180BE1F90EDBCFE9FFDB2AFA0ECD
:100D5000DBCFEAFF01E3DB2A2E0EEF6E060EDBCFC0
:100D60001EF0070EDBCF1FF0F1EC15F00A0E1DC0D0
:100D7000DBFF0B0E1EC0DBFF0C0E1FC0DBFF0D0EDA
:100D800020C0DBFF1DC000F01EC001F01FC002F03C
:100D900020C003F0D950FB0FE96EFF0EDA20EA6E97
:100DA000EECF1DF0EECF1EF0EECF1FF0EFCF20F014
:100DB00000C022F001C023F002C024F003C025F0DF
:100DC0001FEC16F020C0EDFF1FC0EDFF1EC0EDFFB1
:100DD0001DC0EFFF006A016A200E026E410E036E15
:100DE000D950FB0FE96EFF0EDA20EA6EEECF1DF050
:100DF000EECF1EF0EECF1FF0EFCF20F000C022F0BC
:100E000001C023F002C024F003C025F009EC17F064
:100E100020C0EDFF1FC0EDFF1EC0EDFF1DC0EFFFA6
:100E2000040EDB2A050E01E3DB2A3CD7F90EDBCFEB
:100E3000E9FFFA0EDBCFEAFFEF6A0E0EE15C02E299
:100E4000E16AE552E16EE552E7CFD9FF1200D9CF52
:100E5000E6FFE1CFD9FF060EE1260101FE9DFB0E64
:100E6000DBCF1DF0FC0EDBCF1EF0FD0EDBCF1FF045
:100E7000FE0EDBCF20F0A5EC17F01CC0DEFF1DC07E
:100E8000DEFF1EC0DEFF1FC0DDFFDD52DD52FB0EA8
:100E9000DBCF04F0FC0EDBCF05F0FD0EDBCF06F060
:100EA000FE0EDBCF07F0F90EDBCF1EF0FA0EDBCF24
:100EB0001FF0F1EC15F01DC008F01EC009F01FC0B6
:100EC0000AF020C00BF008C022F009C023F00AC0CD
:100ED00024F00BC025F004C01DF005C01EF006C0B4
:100EE0001FF007C020F009EC17F01DC000F01EC075
:100EF00001F01FC002F020C003F0F90EDBCF14F0A8
:100F0000FA0EDBCF15F0166A176A15AE02D0166816
:100F1000176814C01CF015C01DF016C01EF017C0D5
:100F20001FF0DFCF21F0010EDBCF22F0020EDBCF6E
:100F300023F0030EDBCF24F0E7EC1CF018C010F018
:100F400019C011F01AC012F01BC013F010C01CF031
:100F500011C01DF012C01EF013C01FF006EC16F0F9
:100F60001DC00CF01EC00DF01FC00EF020C00FF011
:100F70000CC022F00DC023F00EC024F00FC025F0ED
:100F800000C01DF001C01EF002C01FF003C020F021
:100F90001FEC16F076EC17F0040E1EC0DBFF050EFA
:100FA0001FC0DBFF980EE66E0A0EE66ED9CFE9FF92
:100FB000DACFEAFFEECFE6FFEECFE6FFEECFE6FFB9
:100FC000EFCFE6FF90EC19F0006E060EE15E0050E8
:100FD000980EE66E0A0EE66E24DAE552E552F3CF7D
:100FE000B6F1F4CFB7F12E0EE66EE66A53DAE552AB
:100FF000E552E66A040EDBCFE6FF050EDBCFE6FF27
:101000000DD8E552E552E552060EE15C02E2E16AD6
:10101000E552E16EE552E7CFD9FF1200D9CFE6FFE6
:10102000E1CFD9FF0A0EE12601012D0EE86F010E76
:10103000E96FFC0EDBCF00F0010EE76E0018E8AEA2
:1010400002D0003403D0E750D880005401E2DBD056
:10105000FC0EDB5028E1FD0EDBCF00F0FE0EDBCFF7
:1010600001F0060E00C0DBFF070E01C0DBFF080E1B
:10107000DB6A090EDB6A2D0EE66E010EE66ED950B4
:10108000060FE96EDACFEAFFEECFE6FFEECFE6FF1E
:10109000EECFE6FFEFCFE6FF90EC19F0006E060E04
:1010A000E15E005010D02D0EE66E010EE66EFD0ED4
:1010B000DBCFE6FFFE0EDBCFE6FFF6EC18F0E552E5
:1010C000E552E552E5520101FEAD84D02D0EE66EEB
:1010D000010EE66E1FEC1DF0E552E552020EF3CF55
:1010E000DBFF030EF4CFDBFFDE6ADD6ADECF00F04C
:1010F000DDCF01F0020EDBCF02F0030EDBCF03F0F9
:101100000250005C035001582EE2020EDBCF02F0C9
:10111000030EDBCF03F0DE50025CE96EDD500358B6
:10112000EA6EE906000EEA5A2D0EE926010EEA22C1
:10113000EF50E66EFC0EDB50040F006E016A00BE3D
:101140000168DE50005CE96EDD500158EA6E2D0E3C
:10115000E926010EEA22E552E750EF6EDF2A010E82
:1011600001E3DB2AC3D7DE6ADD6ADECF00F0DDCF24
:1011700001F0FC0EDB50050F046E056A04BE056825
:10118000020EDB50045C026E030EDB500558036E4A
:101190000250005C035001581DE20101FEA90BD072
:1011A000DECFE9FFDDCFEAFF2D0EE926010EEA22B0
:1011B000300EEF6E0AD0DECFE9FFDDCFEAFF2D0E55
:1011C000E926010EEA22200EEF6EDF2A010E01E36E
:1011D000DB2ACBD7FC0EDB50050FE96EEA6AE9BECD
:1011E000EA682D0EE926010EEA22EF6AE8C1E6FF61
:1011F000E9C1E6FF16D9E552E552020EF3CFDBFF57
:10120000030EF4CFDBFF0A0EE15C02E2E16AE55275
:10121000E16EE552E7CFD9FF1200D9CFE6FFE1CF6B
:10122000D9FFE652800EDF6EDF50000821E2DF506A
:10123000F36EFE0EDBCFF4FFF350F45C0FE3310EE0
:10124000E66EE66A27D9E552E552FE0EDB50D880FD
:10125000DF54E76EFE0EE7CFDBFF06D0300EE66E02
:10126000E66A18D9E552E552DF407F0BDF6EDCD726
:10127000E552E552E7CFD9FF1200D9CFE6FFE1CF23
:10128000D9FF020EE126FE0EDB50F00BE8380F0B03
:10129000300FDF6EDF50390803E2070EDF24DF6E08
:1012A000FE0EDB500F0B300FE76E010EE7CFDBFFBA
:1012B000DB5039080AE2070E006E010EDBCFE7FFB4
:1012C0000050E726010EE7CFDBFFDFCFE6FFE66A3F
:1012D000E1D8E552E552010EDBCFE6FFE66ADAD847
:1012E000E552E552680EE66EE66AD4D8E552E5525C
:1012F000020EE15C02E2E16AE552E16EE552E7CFFF
:10130000D9FF12000101005107E1C20E011904E1E9
:10131000010E021901E1035130E0005106E1960E81
:10132000011903E1025101E1035122E0005106E1FC
:101330004B0E011903E1025101E1035114E0800E4B
:10134000001906E1250E011903E1025101E10351E3
:1013500005E0820E0101DD6FDE6B14D0820E01010B
:10136000DD6FDE6B0FD0400E0101DD6FDE6B0AD04A
:10137000200E0101DD6FDE6B05D00A0E0101DD6F6D
:10138000DE6B00D0410EDD6FDE6BDDC1E6FFDEC13E
:10139000E6FF740EE66EAEEC1CF0E552E552E55247
:1013A0009F8AD08E9D9AF29CF29E1200D9CFE6FFC2
:1013B000E1CFD9FF020EE126DE6ADD6AFD0EDBCF4A
:1013C000F6FFFE0EDBCFF7FF0800F55017E0FD0E2D
:1013D000DBCFF6FFFE0EDBCFF7FF0800F550E66E21
:1013E000E66A58D8E552E552DF2A010E01E3DB2A0E
:1013F000FD0EDB2AFE0E01E3DB2AE0D7DECF00F094
:10140000DDCF01F000C0F3FF01C0F4FF020EE15C8C
:1014100003E200D0E16AE552E16EE552E7CFD9FF81
:101420001200D9CFE6FFE1CFD9FF020EE126DE6A36
:10143000DD6AFD0EDBCFE9FFFE0EDBCFEAFFEF50EA
:1014400016E0FD0EDBCFE9FFFE0EDBCFEAFFEF502B
:10145000E66EE66A1FD8E552E552DF2A010E01E387
:10146000DB2AFD0EDB2AFE0E01E3DB2AE2D7DECF0C
:1014700000F0DDCF01F000C0F3FF01C0F4FF020E69
:10148000E15C03E200D0E16AE552E16EE552E7CFAC
:10149000D9FF1200D9CFE6FFE1CFD9FFACA2FED72A
:1014A000FD0EDBCFE6FFE1EC1DF0E552E552E7CFA4
:1014B000D9FF12000D0EE66EE66AECDFE552E5524A
:1014C0000A0EE66EE66AE6DFE552E5521200D9CF73
:1014D000E6FFE1CFD9FFFB0EDBCF1DF0FC0EDBCF2B
:1014E0001EF0FD0EDBCF1FF0FE0EDBCF20F0203410
:1014F000000E201809E6D880000E1D54000E1E5460
:10150000000E1F54000E20540CE2D950FB0FE96E60
:10151000FF0EDA20EA6EEE06000EEE5AEE5AEE5A92
:10152000DAD7E552E7CFD9FF12000F013F8F3F9D79
:101530003F8B3F893F873F853F833F913E8F3E9D55
:101540003E893E873E853E833E813D873D853D8386
:101550003D918168396B93689380938293849386DD
:101560009388938A938C938EF19E6168386B38814F
:10157000388338852F0E926E82683A6BBF0E946E58
:10158000949C948ED08ED09C606A1200CD9ECD9C8F
:10159000CD8ACD88CD9ACD98CD96CD94CD82CD9063
:1015A000CC9ECC9ACC92CC909F80D08EDB0EE66EF7
:1015B0000B0EE66E95EC1DF0E552E5529E90F29C06
:1015C000CD909D90F29EF29C1200AFDF0101FE8D46
:1015D000FE89FE95FE97FC6BFD6BFA6BFB6B8988B1
:1015E000F46BF56B0A01586B0101FE9F8BDE9EAA1E
:1015F00005D076EC1DF00101F36FF9D70101F36B13
:101600000C0EE66EE66A46DFE552E552A00EE66E87
:10161000860EE66E010EE66EE66A59DFE552E55289
:10162000E552E552000EE66EE66A7AEC00F0E5520D
:10163000E552200EE66EE66A7AEC00F0E552E552DD
:10164000400EE66EE66A7AEC00F0E552E5520101E2
:10165000980E3E6F0A0E3F6FF00EE66E490EE66E74
:10166000020EE66EE66A33DFE552E552E552E552D8
:10167000C69A01014E0EDA6F800EE66E080EE66E17
:10168000B1EC1DF0E552E552180EC86EC750040BC0
:1016900001E0010E006E1F0EC514001001E0F6D728
:1016A000C580C5B0FED70101B46BB56BC9CFDBF106
:1016B000DAC1E6FF6EEC1CF0E5520101DC6FFF0EB3
:1016C000DC5D03E1C9CFDBF1C69EB42B000EB52370
:1016D000DC5105E0C80EB45D000EB559E9E3C80E53
:1016E000B45D000EB55920E2B4C1E6FFB5C1E6FF16
:1016F000DA51E66EE66A610E006E350E016E026A20
:1017000000C0E6FF01C0E6FF02C0E6FFFE0EE66E87
:10171000E668DEEC1BF0036E090EE15E0350F3CFCA
:10172000B6F1F4CFB7F122D0B4C1E6FFB5C1E6FF00
:10173000DC51E66EE66ADA51E66EE66A270E006E66
:10174000350E016E026A00C0E6FF01C0E6FF02C06E
:10175000E6FFFE0EE66EE668DEEC1BF0036E0B0E97
:10176000E15E0350F3CFB6F1F4CFB7F1A3DE010190
:101770004E0EDA6F20EC02F00101DC6B010EE66E1A
:10178000E66E77EC01F0E552E552010EE66E020ED0
:10179000E66E77EC01F0E552E55201014E0EDA6F8C
:1017A00020EC02F0100EE66E270EE66EE66AE66AA0
:1017B0008EDEE552E552E552E552010EE66EE66E2A
:1017C00077EC01F0E552E552010EE66E020EE66E90
:1017D00077EC01F0E552E552010EE66E800EE66E02
:1017E00077EC01F0E552E552010EE66EE66AB8ECE0
:1017F00000F0E552E552010EE66EC00EE66E77ECA3
:1018000001F0E552E552020EE66EE66AB8EC00F031
:10181000E552E552010EE66E940EE66E77EC01F0AD
:10182000E552E552030EE66EE66AB8EC00F0E552CA
:10183000E552010EE66ED40EE66E77EC01F0E5524D
:10184000E552040EE66EE66AB8EC00F0E552E552A9
:10185000800EE66E1A0EE66E060EE66EE66A37DE5D
:10186000E552E552E552E5520101FE9F100EE66E8B
:10187000270EE66EE66AE66A2ADEE552E552E55292
:10188000E552020EE66EE66A03EC03F0E552E5521D
:10189000030EE66EE66A03EC03F0E552E552040E31
:1018A000E66EE66A03EC03F0E552E552010EE66EE1
:1018B000800EE66E77EC01F0E552E5520101DF6B38
:1018C000E06BF36B0A01586B0101F46BF56BC2809E
:1018D000C19EC08EC08AC088C096C084C092C0809D
:1018E000C196C194C192C190FE9789884FDE9E90A7
:1018F000F28CF29EF29C9D90CD900101FE95D46BEE
:10190000D56BF66BF76BF36BF86BF96B030EE66E4A
:10191000E66A03EC03F0E552E552040EE66EE66A71
:1019200003EC03F0E552E5520A01586B0101FE9504
:10193000DF6BE06B010EE66EE66A03EC03F0E55246
:10194000E552020EE66EE66A03EC03F0E552E5525C
:10195000030EE66EE66A03EC03F0E552E552040E70
:10196000E66EE66A03EC03F0E552E552A3DD010EF4
:10197000E66EE66A03EC03F0E552E552130E006EE4
:10198000350E016E026A00C0E6FF01C0E6FF02C02C
:10199000E6FF3EC1E6FF3FC1E6FF39EC1BF0036EF8
:1019A000050EE15E0350F3CFB6F1F4CFB7F13EC1BF
:1019B000E6FF3FC1E6FFC9EC02F0E552E5523EC149
:1019C000E6FF3FC1E6FF2DDDE552E552020EE66E71
:1019D000E66A03EC03F0E552E5520101D00ECE6F4A
:1019E000E30ECF6F840ED06F3E0ED16F040EE66E05
:1019F0003EC1E6FF3FC1E6FFCEC1E6FFCFC1E6FF35
:101A0000D0C1E6FFD1C1E6FFC6EC03F0006E070EC1
:101A1000E15E00503EC1E6FF3FC1E6FFC9EC02F0C7
:101A2000E552E5523EC1E6FF3FC1E6FFFADCE55272
:101A3000E55240DD82A23EDD400EE66E0D0EE66E02
:101A4000030EE66EE66A43DDE552E552E552E552E5
:101A50000101C66BC76BC86BC96BCA6BCB6BCC6B18
:101A6000CD6BB86BB96B0101B46BB56BBA6BBB6B6B
:101A70009E90B10EE66E3C0EE66E95EC1DF0E552C2
:101A8000E552CD809EB02BD0010EC26EC280010106
:101A9000BA2B000EBB2358EC1EF053EC1EF00009CD
:101AA00001E0FBD741EC1EF0F3CF00F0F4CF01F0E2
:101AB000B4C1E9FFB5C1EAFF010ED890E936EA36B4
:101AC000E806FBE1000EE926080EEA2200C0EEFF60
:101AD00001C0EDFF0101B42B000EB523D3D7CD908B
:101AE0009E904E0EE66EE66AD5DCE552E5523D0E5E
:101AF000E66EE66ACFDCE552E552E66ABAC1E6FF79
:101B0000BBC1E6FF0EEC08F0E552E552E552090EC6
:101B1000E66EE66ABFDCE552E5524C0EE66EE66A1A
:101B2000B9DCE552E5523D0EE66EE66AB3DCE552FD
:101B3000E552E66AB8C1E6FFB9C1E6FF0EEC08F06F
:101B4000E552E552E552090EE66EE66AA3DCE5527F
:101B5000E55282A2AFDC0101BC6B040EBD6FBE6B0F
:101B6000BF6BB46BB56BBA51B45DBB51B5593FE2B5
:101B7000B4C1E9FFB5C1EAFF010ED890E936EA36F3
:101B8000E806FBE1000EE926080EEA22EECFD6F1C8
:101B9000EDCFD7F10101BC51D65DBD51D75904E25B
:101BA000D6C1BCF1D7C1BDF1D651BE5DD751BF5929
:101BB00004E2D6C1BEF1D7C1BFF182B213D0FE8D0F
:101BC000E66AD6C1E6FFD7C1E6FF0EEC08F0E552A3
:101BD000E552E5520101FE9D3B0EE66EE66A5ADCD7
:101BE000E552E5520101B42B000EB523BCD782B2F9
:101BF00002D060DC06D0090EE66EE66A4BDCE552E8
:101C0000E552010EE66EE66A03EC03F0E552E5529A
:101C1000B8C1E6FFB9C1E6FFFE0E006E340E016EDC
:101C2000026A00C0E6FF01C0E6FF02C0E6FF3EC157
:101C3000E6FF3FC1E6FF39EC1BF0036E070EE15EE5
:101C40000350F3CFB6F1F4CFB7F13EC1E6FF3FC189
:101C5000E6FFC9EC02F0E552E5520101BC51BE5D60
:101C6000C06FBD51BF59C16FC0C1E6FFC1C1E6FF22
:101C7000BCC1E6FFBDC1E6FFBEC1E6FFBFC1E6FFD6
:101C8000D70E006E340E016E026A00C0E6FF01C07E
:101C9000E6FF02C0E6FFFE0EE66EE668DEEC1BF035
:101CA000036E0B0EE15E0350F3CFB6F1F4CFB7F144
:101CB000BCC1E6FFBDC1E6FFBEC1E6FFBFC1E6FF96
:101CC000C20E006E340E016E026A00C0E6FF01C053
:101CD000E6FF02C0E6FF3EC1E6FF3FC1E6FF39EC8A
:101CE0001BF0036E090EE15E0350F3CFB6F1F4CFA3
:101CF000B7F1020EE66EE66A03EC03F0E552E55238
:101D00003EC1E6FF3FC1E6FFC9EC02F0E552E552F5
:101D1000C0C1E6FFC1C1E6FFB00E006E340E016E19
:101D2000026A00C0E6FF01C0E6FF02C0E6FF3EC156
:101D3000E6FF3FC1E6FF39EC1BF0036E070EE15EE4
:101D40000350F3CFB6F1F4CFB7F1030EE66EE66AB7
:101D500003EC03F0E552E5523EC1E6FF3FC1E6FF6A
:101D6000C9EC02F0E552E552C0C11EF0C1C11FF03E
:101D7000EFEC15F01DC000F01EC001F01FC002F016
:101D800020C003F0CEC122F0CFC123F0D0C124F097
:101D9000D1C125F000C01DF001C01EF002C01FF02F
:101DA00003C020F009EC17F01DC0C2F11EC0C3F142
:101DB0001FC0C4F120C0C5F1C2C122F0C3C123F0CD
:101DC000C4C124F0C5C125F0CAC11DF0CBC11EF0AD
:101DD000CCC11FF0CDC120F020EC16F01DC0CAF11F
:101DE0001EC0CBF11FC0CCF120C0CDF1040EE66EB9
:101DF000E66A03EC03F0E552E5520101B82B000E50
:101E0000B923090ED880B855000EB95501E379D031
:101E1000226A236A200E246E410E256ECAC11DF06F
:101E2000CBC11EF0CCC11FF0CDC120F0B6EC16F036
:101E30001DC0C6F11EC0C7F11FC0C8F120C0C9F146
:101E4000A50E006E340E016E026A00C0E6FF01C0EE
:101E5000E6FF02C0E6FF3EC1E6FF3FC1E6FF39EC08
:101E60001BF0036E050EE15E0350F3CFB6F1F4CF25
:101E7000B7F13EC1E6FF3FC1E6FFC9EC02F0E55213
:101E8000E5523EC1E6FF3FC1E6FF11EC0AF0E55224
:101E9000E552020EE66E3EC1E6FF3FC1E6FFC6C157
:101EA000E6FFC7C1E6FFC8C1E6FFC9C1E6FFC6EC51
:101EB00003F0006E070EE15E00503EC1E6FF3FC139
:101EC000E6FFC9EC02F0E552E5523EC1E6FF3FC134
:101ED000E6FF11EC0AF0E552E5520101CA6BCB6B4B
:101EE000CC6BCD6BB86BB96B500EE66EC30EE66E65
:101EF000E66AE66A67EC0AF0E552E552E552E55219
:101F00004DD09A0E006E340E016E026A00C0E6FFDC
:101F100001C0E6FF02C0E6FF3EC1E6FF3FC1E6FFAB
:101F200039EC1BF0036E050EE15E0350F3CFB6F102
:101F3000F4CFB7F13EC1E6FF3FC1E6FFC9EC02F0C6
:101F4000E552E5523EC1E6FF3FC1E6FF11EC0AF063
:101F5000E552E552010EE66E3EC1E6FF3FC1E6FFE7
:101F6000C2C1E6FFC3C1E6FFC4C1E6FFC5C1E6FFCB
:101F7000C6EC03F0006E070EE15E00503EC1E6FFC6
:101F80003FC1E6FFC9EC02F0E552E5523EC1E6FF73
:101F90003FC1E6FF11EC0AF0E552E552300EE66E65
:101FA000750EE66EE66AE66A67EC0AF0E552E552FF
:101FB000E552E5525AEC0AF056D512001AEC15F02B
:101FC000FB0EDBCFF3FFDB06F35000090AE068EC01
:101FD00015F0FA0ED3EC15F0F3E1011CF1E1010E5E
:101FE00001D0000E49EF15F01AEC15F03B0EE1247C
:101FF00002E3E168E652E16E010EDB6A020EDB6A83
:10200000F90EDBCFF6FFFA0EDBCFF7FFFB0EDBCFCF
:10201000F8FF0800F550DF6EDF5002E16DEF14F0BD
:10202000250EDF5C02E060EF14F0030EDB6A040EA5
:10203000DB6A050EDB6A060EDB6A070EDB6A82ECE2
:1020400014F02D0EDF5C0CE02B0EDF5C09E0200E9F
:10205000DF5C06E0230EDF5C03E0300EDF5C1AE19C
:10206000DF50300A14E0130A0FE0030A0AE00B0AFB
:1020700005E0060AE4E1030EDB80E1D7030EDB8214
:10208000DED7030EDB84DBD7030EDB86D8D7030E47
:10209000DB88D5D72A0EDF5C1BE17EEC14F0CCEC9C
:1020A00014F010E0030EDB801E681F68130EDBCFF8
:1020B00023F0140EDBCF24F0C9EC18F0040E1CC082
:1020C000DBFF03D0130EB5EC14F082EC14F00BD050
:1020D000090EDB6A23EC15F003E097EC15F0FAD754
:1020E000090EB5EC14F0030EDBB0DB982E0EDF5CAE
:1020F0001BE182EC14F02A0EDF5C0BE17EEC14F0A5
:10210000CCEC14F003E1130E07EC15F082EC14F0A4
:102110000BD0090EDB6A23EC15F003E097EC15F009
:10212000FAD7090E07EC15F0680EDF5C07E182ECC8
:1021300014F0680EDF5C1DE1030E18D0740EDF5C36
:1021400017E07A0EDF5C14E0480EDF5C06E0540E08
:10215000DF5C03E05A0EDF5C02E1020E07D06C0E7A
:10216000DF5C03E06A0EDF5C04E1010E5AEC15F05F
:10217000C9DBDF506E0A01E17FD31E0A01E192D173
:10218000200A01E18FD13F0A01E149D11A0A01E198
:1021900046D10D0A01E143D1200A01E140D13A0ABA
:1021A00001E13DD1200A01E13AD1260A01E135D110
:1021B0000D0A01E132D11A0A01E1D9D0200A4AE020
:1021C000300A1FE0460A0EE0250A01E083D3D95009
:1021D000F90FE96EFF0EDA20EA6E010EEE5E000ED8
:1021E000EE5AEE5A68EC15F0250EE66E95DB03E12B
:1021F000011C01E169D364EC15F001E26BD3DB2A29
:1022000069D3080EDB6A040EDB50010806E2040EF7
:10221000DB042CEC15F0DB508BDB080EDB5009E007
:10222000030EDB50010B05E172DB01E04DD3080E1C
:10223000DB6A64DBEFCFDFFFDCEC15F003E1011CB0
:1022400001E142D364EC15F001E3DB2A60DB01E13C
:1022500041D33AD3070EDB5002080FE1A8EC15F08A
:10226000030E6FEC15F00E0EEECFDBFF0F0EEECF70
:10227000DBFF100EEECFDBFF20D0F70EDBCF03F03D
:10228000F80EDBCF04F0020E035E000E045AF70EC8
:1022900003C0DBFFF80E04C0DBFF03C0E9FF04C08E
:1022A000EAFF5FEC15F0026A0E0E00C0DBFF0F0EB6
:1022B00001C0DBFF100E02C0DBFF0E0EDBCFE6FF1E
:1022C0000F0EDBCFE6FF100EDBCFE6FF2DEC1DF08F
:1022D000E552E552E552130E1DC0DBFF140E1EC081
:1022E000DBFF060EDB5005E0130EA3EC15F001E258
:1022F0006ADBC7EC15F002E2130E37DB8AEC15F04F
:1023000006E0040EA3EC15F002E2050E2EDB030E30
:10231000DBB005D0FCDA01E0D7D2080EDB6A090E8B
:10232000DB6A0E0EDBCFF6FF0F0EDBCFF7FF100ED2
:10233000DBCFF8FF0800F550DF6EDF5014E0CDEC86
:1023400015F011E2DCEC15F003E1011C01E1BCD257
:10235000BBDB01E3DB2A090EDB2AD9500E0FE96E45
:10236000000ECBDBE7D7D3DA01E1B4D2ADD2C6DAC7
:10237000110EEECFDBFF120EEDCFDBFF110EDBCF28
:10238000E6FF120EDBCFE6FF1FEC1DF0E552E55233
:10239000130EF3CFDBFF140EF4CFDBFF060EDB5082
:1023A00004E0130ED0DB01E20EDBC7EC15F002E215
:1023B000130EDBDAAFDB05E0040EC5DB02E2050E2F
:1023C000D4DA030EDBB005D0A2DA01E07DD2080E2C
:1023D000DB6A090EDB6A110EDBCFE9FF120EDBCFE1
:1023E000EAFFEFCFDFFFDF5014E0D7DB12E2E4DBE0
:1023F00003E1011C01E168D267DB01E3DB2A090E7E
:10240000DB2A110EDB2ADBCFE9FF120EE8E3DB2A21
:10241000E6D77DDA01E15ED257D2030EDB8E070EDE
:10242000DB0410E195DB040E5ADB0A0EEECFDBFF76
:102430000B0EEECFDBFF0C0EEECFDBFF0D0EEECF63
:10244000DBFF6CD0070EDB5003082CE1030EDBAE84
:102450000DD0B2DA020E76DAEFCF00F0016A026A2E
:10246000036A00AE39D00168026835D0F70EDBCFC1
:1024700001F0F80EDBCF02F0020E015E000E025AF0
:10248000F70E01C0DBFFF80E02C0DBFF01C0E9FF61
:1024900002C0EAFFEFCF00F00A0E00C0DBFF0B0E18
:1024A000DB6A38D0070EDB50020809E1030EDBAE11
:1024B00004D059DB02AE10D00ED055DB0DD0030E88
:1024C000DBAE12D079DA020E3DDAF9DA026A036A7B
:1024D00001AE02D002680368E2DA0C0E02C0DBFF34
:1024E0000D0E03C0DBFF1AD0F70EDBCF02F0F80EA3
:1024F000DBCF03F0020E025E000E035AF70E02C09D
:10250000DBFFF80E03C0DBFF02C0E9FF03C0EAFFF8
:10251000D6DAC5DA0C0EDB6A0D0EDB6A060EDB506E
:1025200005E1010EF36E050EF3CFDBFF150EDB6A3E
:10253000160EDB6AD950370F006E000EDA20016EDE
:10254000390E00C0DBFF3A0E01C0DBFF380EDB6A3C
:10255000080EDB6A0A0EAEDADF50780A12E0200AB3
:1025600010E0280A0CE0200A0AE03F0A06E00D0A03
:1025700002E0200A08E1020E05D0080E03D0080E82
:10258000DF26100E97DA030EDBBE02D0DB92DB945F
:10259000DB50800B24E08ADAD890030EEB50000A5F
:1025A00008E6000EEE5C000EEE58000EEE58000E2F
:1025B000EE5815E213DA2168226823682468E7ECF4
:1025C0001CF00A0E18C0DBFF0B0E19C0DBFF0C0E4F
:1025D0001AC0DBFF0D0E1BC0DBFF2D0E08D0030E53
:1025E000DBA202D02B0E03D0DBA408D0200EF36EAA
:1025F000170EF3CFDBFF150EDB2A02D0170EDB6AB6
:10260000050EDB5003E1B7D901E189D0940E006ECD
:102610003C0E016E000E026E070EDBCF03F0046A63
:10262000056A066A03C021F004C022F005C023F049
:1026300006C024F0D3D952EC1DF000501824F36EDC
:1026400001501920F46E02501A20F86EF4CFF7FFF3
:10265000F3CFF6FF0800090EF5CFDBFF580EDF5C65
:102660000FE1610EF36E090E7BD90AE3200E006EB6
:10267000090EDBCFE7FF0050E75E090EE7CFDBFF77
:10268000070EDBCF00F0016A026A036A0FDA00C0AE
:1026900021F001C022F002C023F003C024F0EECFED
:1026A0001CF0EECF1DF0EECF1EF0EFCF1FF052EC7E
:1026B0001DF01FC0EDFF1EC0EDFF1DC0EDFF1CC0D3
:1026C000EFFF390EDBCFE9FFDB063A0EDBCFEAFF87
:1026D00001E2DB06090EDBCFEFFF150EDB2A4BD93B
:1026E00095E1030EDBA61DD06F0EDF5C06E1C1D9BC
:1026F00018E3150EDB285BDA14D0780EDF5C09E0F6
:10270000580EDF5C06E0620EDF5C03E0420EDF5C29
:1027100008E1020EF36E160EF3CFDBFF02D0150EAA
:10272000DB6A030EDB50100B0EE0040EDBCF00F073
:10273000050EDB50D880005406E2060EDB5003E1A4
:10274000040EDB5034DA95D90AE2050EDBCFE7FF41
:10275000150EDB50E75E050EE7CFDBFF02D0050E5E
:10276000DB6A040EDBCF00F0160E45D9D88000548A
:1027700014E2160EDBCFE6FF150EDBCFE6FF040EEC
:10278000DBCFE6FF050EDB50E552E75CE552D88073
:10279000E754E552D880E7545FD9030EDB50010BB4
:1027A0000BE1080EDB5008E0B2D801E08DD0080E36
:1027B000DB50BED8080EDB6A170EDB5007E088D965
:1027C000170EF1D903E1011C01E17ED0160EDB509A
:1027D00016E07ED9300EE66E9FD802E1011C74E04F
:1027E00077D9DFCFE6FF2CEC1CF0E552E552E5523D
:1027F000F4CF01F00001F31C02E1011C65E0050EBD
:10280000DBCF00F0160EDB50D880005409E2050E35
:10281000DBCFE7FF160EDB50E75E050EE7CFDBFFF1
:10282000300EE66E050ECBD94FE1390EDB2ADBCF39
:10283000E9FF3A0E01E3DB2ADBCFEAFF090EEFCF17
:10284000DBFFDB500EE044D9090EADD902E1011CDB
:102850003BE0390EDB2ADBCFE9FF3A0EEDE3DB2A62
:10286000EBD755D831E1160EDBCFE6FF080EC3D803
:10287000E552E7245DD82ED0070EDB50030A1CE09A
:10288000010A14E0030A07E07BD9DBCFEEFF020E5A
:10289000DBCFEDFF1FD0F5D8056A03AE02D0046888
:1028A00005682CD8BCD805C0EEFF14D0EAD803BE0A
:1028B000046824D8B4D80ED063D9DBCFEFFF0AD098
:1028C0007BD905E1011C03E1F368F46810D0FCD862
:1028D00001E3DB2A79D909EF10F0010EDBCF00F01C
:1028E000020EDBCF01F000C0F3FF01C0F4FF3B0E8E
:1028F000E15C02E2E16AE552E16ECBD029D9020E39
:102900006FEF15F061D90800F550DF6E1200200E50
:10291000E66E080EDFEF15F02CEC1CF0E552E552E8
:10292000E552F3CF00F0F4CF01F00001F31C1200E8
:10293000006E016AD950010F4DD90050EE260150AA
:10294000ED221200045E000E055AF70E04C0DBFFF4
:10295000F80E05C0DBFF04C0E9FF05C0EAFF120066
:10296000DBCFF4FFF350F45C1200DB50E76E040E93
:10297000E7CFDBFF12000A0EDBCF00F00B0EDBCF40
:1029800001F00C0EDBCF02F00D0EDBCF03F0005098
:102990000110021003101200130EEECFDBFF140E15
:1029A000EDCFDBFF130EDBCF00F0140EDBCF01F019
:1029B0000001800E01141200F70EDBCF04F0F80EB8
:1029C000DBCF05F01200050EDB50E66ED950130F79
:1029D00001D9E552E750EE6EED6A12000A0EDBCF28
:1029E0001CF00B0EDBCF1DF00C0EDBCF1EF00D0E1E
:1029F000DBCF1FF01200DBCFE6FF150EDBCFE6FFCB
:102A0000050EDB50E552E724E552E7241200DB50C7
:102A1000CED8010EF36E060EF3CFDBFF1200EE50A0
:102A2000EFCFEAFFE96E02C0EEFF03C0EEFF04C085
:102A3000EEFF1200D9CFE6FFDACFE6FFE1CFD9FFF4
:102A4000E2CFDAFF1200DFCFE6FFE66AF8EC1DF016
:102A5000E552E552F3501200E76E080EE7CFDBFFB8
:102A60001200EECF00F0EECF01F0EFCF02F0036ADC
:102A70001200050EDBCF00F0150EDB50D88000549D
:102A80001200010EDBCF02F0020EDBCF03F0046A6E
:102A90001200E552E5CFDAFFE7CFD9FF12000A0EA8
:102AA00000C0DBFF0B0E01C0DBFF1200D9500A0F84
:102AB000EAEF15F0F36E070EF3CFDBFF1200EECF57
:102AC00000F0EFCF01F01200010EDB2A020E12001F
:102AD000FC0EDBCFE6FFFD0EDBCFE6FF1200005E53
:102AE000000E015AF70E00C0DBFFF80E01C0DBFF3D
:102AF00000C0E9FF01C0EAFF1200DA20EA6EEF2A07
:102B0000EECFF6FF000EEF22EECFF7FFEF22EECF73
:102B1000F8FF1200040EDBCFE6FF130EDB50E55288
:102B2000E75C9ADFDB5004DF060EDB501200090E73
:102B3000DB500A0DF350DF24D00FE76E090EE7CF0C
:102B4000DBFF82EF14F0DB50F36E050EB0EF14F0F4
:102B5000F70EDBCF00F0F80EDBCF01F01200DFCF75
:102B6000E6FF8CEF14F028DF030EECDE31EF15F0FA
:102B7000DEEC0FF0E552E552E552E5520009120095
:102B8000BDDEEE50EFCFEAFFE96E010E1200130E2C
:102B9000DB50F36E040EB0EF14F0040EDB50F36E56
:102BA000090EB0EF14F0DBCFE6FF8CEF14F0E76E08
:102BB000050EE7CFDBFF12008BDFAFEF15F0DBCFA9
:102BC000E6FF86DFB8EF15F0D950F90FE96EFF0E7A
:102BD0007DEF15F0E96E000EDA20EA6E1200279EF6
:102BE00008D0279E1FAE05D01E6C1F1EE86A1F224C
:102BF000278E1FC019F01EC018F02B6A2A6A8E0E8D
:102C00001A6E1B6A5FEF18F0279E0CD0279E1FAE2E
:102C100009D01C6C1D1E1E1E1F1EE86A1D221E22CE
:102C20001F22278E1FC019F01EC018F01DC02BF0E8
:102C30001CC02AF09E0E1A6E1B6A5FEF18F0257EEC
:102C4000276A9BEC18F0B3EC18F027B643EF18F0A6
:102C500027A20AD027AA03D027BE43EF18F027A443
:102C60004FEF18F04CEF18F027AA05D027AC4FEF24
:102C700018F04CEF18F027A00AD027A808D027BEDC
:102C800004D027A402D058EF18F05CEF18F02A6A9D
:102C90001B6A2550205C296E10E31DC02BF01EC05E
:102CA00018F01FC019F020C028F022C01DF023C06A
:102CB0001EF024C01FF0273A09D022C02BF023C0F9
:102CC00018F024C019F025C028F0296C279E27BCD5
:102CD000278E28C01AF027B08BEF18F01A0E296043
:102CE0008BEF18F01A6A206A27A408D01D6C1E1EEC
:102CF0001F1E201EE86A1E221F22202227AC08D099
:102D00002B6C181E191E1A1EE86A182219221A2284
:102D10001C6A295207E020341F321E321D321C3239
:102D2000292EF9D71D502B261E5018221F5019226C
:102D300020501A221CC02AF0279E1AAE0BD02A6CF3
:102D40002B1E181E191E1A1EE86A2B221822192281
:102D50001A22278E1AA006D0D880193218322B32A8
:102D60002A32282A28C01AF05FEF18F0276A9BEC55
:102D700018F0B3EC18F027B643EF18F027A205D0EF
:102D800027BA43EF18F04AEF18F027BA56EF18F0B9
:102D900027A005D027B843EF18F056EF18F027B852
:102DA0004AEF18F01B6A7F0E20241A6EE86A1B2275
:102DB00025501A5EE86A1B5A1A0E286E206A2A6A83
:102DC0002B6A186A196A22501D5E23501E5A24501D
:102DD0001F5A000E205A09E722501D2623501E229A
:102DE00024501F22000E202201D02A8AD8901D369E
:102DF0001E361F362036D8902A362B36183619360E
:102E0000282EE1D71F501E101D10D8A42A8A5FEF6C
:102E100018F0276A9BEC18F0B3EC18F027B643EFD4
:102E200018F027A205D027B843EF18F04AEF18F0A2
:102E300027AA05D027B043EF18F04AEF18F027B0C3
:102E400002D027A802D056EF18F01B6A2550202484
:102E50001A6EE86A1B227E0E1A5EE86A1B5A2A6AFC
:102E60002B6A186A196A24501F02F4CF19F0F3CFA5
:102E700018F023501F02F3502B26F4501822000E96
:102E8000192224501E02F3502B26F4501822000E53
:102E9000192222501F02F3502A26F4502B22000E32
:102EA0001822192223501E02F3502A26F4502B22F6
:102EB000000E1822192224501D02F3502A26F45025
:102EC0002B22000E1822192222501E02F4502A260C
:102ED000000E2B221822192223501D02F4502A26FC
:102EE000000E2B22182219225FEF18F0276A9BECA4
:102EF00018F027B680EF17F027A20ED027B405D020
:102F00007F0E1F6EFF0E1E6E1FD0800E1F6E1E6A7C
:102F10001BD01F6A1E6A18D027B0FBD78F0E206007
:102F2000EDD77E0E2064F5D78E0E205C05E0D8909C
:102F30001F321E32202AF8D727A406D01E6C1F1E6F
:102F4000E86A1F221FAEE5D71200276A9BEC18F033
:102F500027B6AFEF17F027A20FD027B407D07F0E08
:102F60001F6EFF0E1E6E1D6E1C6E25D0800E1F6E16
:102F700001D01F6A000EF6D727B0FBD71C6A9F0E40
:102F80002060EBD77E0E2064F4D79E0E205C07E015
:102F9000D8901F321E321D321C32202AF6D727A4A9
:102FA0000AD01C6C1D1E1E1E1F1EE86A1D221E223A
:102FB0001F221FAEDED71200EEEC17F027B6000C72
:102FC00027B0000C27B4000C010CEEEC17F027B66C
:102FD000000C27B0000C27A4000C010C276A9BEC06
:102FE00018F0B3EC18F027B6120027AE08D027A0CF
:102FF00004D027A802D02780120027901200255065
:10300000205C0BE124501F5C08E123501E5C05E1AD
:1030100022501D5C02E127801200D8A002D0278E2A
:1030200010D0205025C020F0256E1F5024C01FF066
:10303000246E1E5023C01EF0236E1D5022C01DF0B2
:10304000226E2550205C10E0FF0F09E0279027B486
:1030500003D027AE2784120027AE27941200252A1A
:10306000D89024322332223222501D5E23501E5A21
:1030700024501F5A1FBEEAD7D8901D361E361F3661
:10308000202EF8D7C8D77F0E206EFF0E1F6E1E6E43
:103090001D6E12007F0E27BEFF0E206E02D07F0E27
:1030A000206E800E1F6E1E6A1D6AF3D727AE04D0F5
:1030B000800E206E1F6AF7D7206A1F6AF4D7195056
:1030C00018102B102A10F8E01BBEF0D719BE0CD038
:1030D0001A501B10EBE0D8902A362B3618361936CA
:1030E0001A06D8A01B06F2D71B50D4E11A28D2E04A
:1030F0002AAE11D07F0E2A1402E12BA00CD02B2A6D
:10310000E86A1822192207E3D880193218322B32C4
:103110001A2A1A28BFE01A50C9E02BC01DF018C0A7
:103120001EF019341F6E1A30206E1F32209E27BEEB
:10313000208E49EF18F01F36203602E32784277EC1
:1031400006E12780206A1F6A1E6A1D6A1200202875
:1031500003E0D8801F321200D8901F3202E127828C
:103160001200278612002436253602E3278C277E9C
:1031700006E12788256A246A236A226A1200252824
:1031800003E0D88024321200D8902432EAE1278A62
:1031900012001FC02BF01EC02AF01E502302F4CFD5
:1031A0001DF0F3CF1CF01F502402F4CF1FF0F3CF1B
:1031B0001EF02302F3501D26F4501E22E86A1F223F
:1031C0002A502402F3501D26F4501E22E86A1F22C2
:1031D00024AEEFEF18F02A501E5E2B501F5A2BAE74
:1031E000000C23501E5E24501F5A000CD9CFE6FF5E
:1031F000DACFE6FFFA0EE3CFD9FFFB0EE3CFDAFF1B
:10320000FD0EE35209E72D0EDE6EFC0EE31EE32AEF
:10321000FD0ED8B4E306E31EE652E652E652FD0E7A
:10322000E124E76EFF0EE220E46EE652F70EE3CFF4
:10323000E6FFF70EE3CFE6FF66EC19F0F90EE124A6
:10324000E96EFF0EE220EA6E56EC19F00AE153EC4B
:1032500019F009E156EC19F008E153EC19F007E117
:1032600008D061EC19F05CEC19F061EC19F05CEC41
:1032700019F061EC19F0DE6AF90EE126FF0EE22288
:10328000FF0EE3CFDAFFE552FF0EE3CFD9FFE552A1
:10329000FC0EE124E96EFF0EE220EA6EEECFF3FFB2
:1032A000EFCFF4FF1200EF380F0B1200EF500F0BAF
:1032B00002E1EE52D8841200EF380F0B300FDE6EB1
:1032C0001200EE500F0B300FDE6E1200FC0EE3CF3B
:1032D000E9FFFD0EE3CFEAFF100EE66EEE6AEE6A3E
:1032E000EF6AD890FD0EE336FE0EE336ED36ED368E
:1032F000EF36FF0EE30609E087EC19F0EE5287EC9B
:1033000019F0EE5287EC19F0EDD7E56E1200030EBE
:10331000EF24E8B6EF6E300EEF24E8BEEF6E000C3F
:10332000D9CFE6FFDACFE6FFF80EE3CFD9FFF90EEB
:10333000E3CFDAFFE652E652E652E652E652FB0EE1
:10334000E124E76EFF0EE220E46EE652F30EE3CFD7
:10335000E6FFF30EE3CFE6FFF30EE3CFE6FFF30E57
:10336000E3CFE6FF15EC1AF0F50EE124E96EFF0E4F
:10337000E220EA6E02EC1AF019E105EC1AF018E10D
:1033800002EC1AF017E105EC1AF016E102EC1AF063
:1033900015E105EC1AF014E102EC1AF013E105EC6A
:1033A0001AF012E102EC1AF011E112D00BEC1AF053
:1033B00010EC1AF00BEC1AF010EC1AF00BEC1AF0FF
:1033C00010EC1AF00BEC1AF010EC1AF00BEC1AF0EF
:1033D00010EC1AF0DE6AF50EE126FF0EE222FF0E77
:1033E000E3CFDAFFE552FF0EE3CFD9FFE552FA0E45
:1033F000E124E96EFF0EE220EA6EEECFF3FFEFCF9D
:10340000F4FF1200EF380F0B1200EF500F0B02E128
:10341000EE52D8841200EF380F0B300FDE6E120020
:10342000EE500F0B300FDE6E1200FA0EE3CFE9FF05
:10343000FB0EE3CFEAFF200EE66EEE6AEE6AEE6A5E
:10344000EE6AEF6AD890FB0EE336FC0EE336FD0E13
:10345000E336FE0EE336ED36ED36ED36ED36EF367D
:10346000FF0EE3060FE044EC1AF0EE5244EC1AF0C3
:10347000EE5244EC1AF0EE5244EC1AF0EE5244ECE8
:103480001AF0E1D7E56E1200030EEF24E8B6EF6EF6
:10349000300EEF24E8BEEF6E000C566F6C7461675F
:1034A00065203D20004176657261676520563D00CC
:1034B000456361727420706B32706B203D2530342F
:1034C00064004D6178693D2530346420204D696E7B
:1034D000693D25303464004D6178693D25303464A0
:1034E00020204D696E693D2530346420205065618F
:1034F0006B325065616B3D253034642009004D65A9
:1035000073757265205520736563742E20232530F2
:10351000326400436F6566662043616C6962726164
:1035200074696F6E203D0050422061647265737350
:1035300061676520253032582C20496E6974204916
:10354000324320494E636F72726563746520537411
:10355000617475733D25336420206A3D2535640D03
:1035600000496E6974205043463835373420636F04
:1035700072726563746520416472657373653D257D
:10358000303258206A3D2533640D004672616D6506
:1035900020457272657572206574204F766572667B
:1035A0006C6F7720646574656374696F6E203A2070
:1035B00000506F727420636F6D6D202E2E2E2E2E94
:1035C0002E206264732C206F7576657274200D0A4C
:1035D0000031384632364B32325F4D657375726555
:1035E0005F736563746575725F3530487A5F313338
:1035F000303931372E630D0A0045534320706F7503
:103600007220736F727469720D004A3D2000496E1A
:10361000697420425420466F726365652028656E88
:103620002061766575676C65290D0A0020202020D1
:10363000202020202020202020202020202020208A
:10364000004C696E6B2054696D656F757420457808
:103650006365656420333220736563200D0A00447E
:1036600061792000486F757220004D696E75746530
:103670002000D9CFE6FFDACFE6FFE1CFD9FFE2CFD6
:10368000DAFFE652E652E652E652D950F90F006EE2
:10369000FF0EDA20016E020E00C0DBFF030E01C038
:1036A000DBFF020EDBCFE6FF030EDBCFE6FFF90EFA
:1036B000DBCFE6FFFA0EDBCFE6FFFB0EDBCFE6FF4C
:1036C000D950FC0FE66EFF0EDA20E66EF4EC0FF038
:1036D000006E070EE15C02E2E16AE552E16E005025
:1036E000F3CFDEFFF4CFDDFFFC0EDBCFE9FFFD0EF5
:1036F000DBCFEAFFEF6ADECF00F0DDCF01F000C0E4
:10370000F3FF01C0F4FF040EE15C02E2E16AE5525E
:10371000E16EE552E5CFDAFFE7CFD9FF1200060EE2
:10372000F66E000EF76E000EF86E0F010900F550F0
:10373000056F0900F550066F03E1056701D03DD024
:103740000900F550006F0900F550016F0900F550B0
:10375000026F09000900F550E96E0900F550EA6EA4
:10376000090009000900F550036F0900F550046FC6
:1037700009000900F6CF07FFF7CF08FFF8CF09FFD0
:1037800000CFF6FF01CFF7FF02CFF8FF0F01035381
:1037900002E1045307E00900F550EE6E0307F8E27A
:1037A0000407F9D707CFF6FF08CFF7FF09CFF8FFD7
:1037B0000F010507000E065BBFD71200D9CFE6FF49
:1037C000DACFE6FFE1CFD9FFE2CFDAFFE652E652E9
:1037D000E652E652D950F90F006EFF0EDA20016E64
:1037E00000C0DEFFDD6EDECFE6FFDDCFE6FFF90EC7
:1037F000DBCFE6FFFA0EDBCFE6FFFB0EDBCFE6FF0B
:10380000FC0EDBCFE6FFFD0EDBCFE6FFF4EC0FF0A6
:10381000006E070EE15C02E2E16AE552E16E0050E3
:10382000020EF3CFDBFF030EF4CFDBFF020EDBCF84
:1038300000F0030EDBCF01F000C0F3FF01C0F4FF86
:10384000040EE15C02E2E16AE552E16EE552E5CF89
:10385000DAFFE7CFD9FF1200D9CFE6FFDACFE6FFD4
:10386000E1CFD9FFE2CFDAFFFB0EDBCF00F0FC0E99
:10387000DBCF01F00001800E01141AE1FB0EDBCF5B
:10388000E9FFFC0EDBCFEAFFEECFF3FFEDCFF4FF55
:10389000EE2A000EEF22F3CFE9FFF4CFEAFFFD0E90
:1038A000DBCFEFFFEF50016AF36E01C0F4FF10D0E1
:1038B000FB0EDB50FE0806E1FD0EDBCFE6FF28EC39
:1038C0001EF005D0FD0EDBCFE6FF5AEC1EF0E552F0
:1038D000E552E5CFDAFFE7CFD9FF1200D9CFE6FFF7
:1038E000DACFE6FFE1CFD9FFE2CFDAFFFD0EDB5002
:1038F000C96EC6AE02D0FF0E2BD00F0EC61408083C
:103900000FE00F0EC6140B080BE0C6889EA6FED76C
:10391000C750040B03E1C750010B17E0000E18D08D
:103920000F0EC614080804E00F0EC6140B0810E1B1
:10393000C7B0FED7C750040B01E0010E006E1F0E8A
:10394000C5140010F7E1C5AC02D0FE0E01D0000E88
:10395000E552E5CFDAFFE7CFD9FF1200D9CFE6FF76
:10396000DACFE6FFE1CFD9FFE2CFDAFFAC6AAB6A8C
:10397000FD0EDBB0AC88DBA202D0AC8CAB8CDBB430
:10398000AC8EDBA602D0AB8801D0AB8ADBB8AC84AE
:10399000DBBAAB86DBAC02D09D8A01D09D9ADBAE50
:1039A00002D09D8801D09D98FB0EDB50AF6EFC0EBF
:1039B000DBCF01F001C000F0016A0050B06EAC8AAC
:1039C000AB8EE552E5CFDAFFE7CFD9FF12001C50EE
:1039D0002102F3CF18F0F4CF19F02202F350192688
:1039E000000EF4201A6E1C502302F3501A26000E0B
:1039F000F4201B6E1C502402F3501B261D50210284
:103A0000F3501926F4501A22000E1B221D502202D8
:103A1000F3501A26F4501B221D502302F3501B268C
:103A20001E502102F3501A26F4501B221E5022026F
:103A3000F3501B261F502102F3501B261200FE0ECE
:103A4000E3CFE9FFFF0EE3CFEAFFF36AF46AEE5239
:103A500003E0F34AF42AFBD71200FF0EE3CFF8FF8E
:103A6000E552FF0EE3CFF7FFE552FF0EE3CFF6FF7F
:103A7000E552E66AE66AE66A0900F55209E0FD0EDB
:103A8000E32A05E1FE0EE32A02E1FF0EE32AF4D762
:103A9000FD0EE3CF1DF0FE0EE3CF1EF0FF0EE3CFD1
:103AA0001FF012001B6A1A6A196A186A200EE76E64
:103AB000D8901C361D361E361F36183619361A3663
:103AC0001B362150185C2250195823501A58245084
:103AD0001B5809E32150185E2250195A23501A5AD4
:103AE00024501B5A1C2AE72EE4D71200D9CFE6FF38
:103AF000DACFE6FFE1CFD9FFE2CFDAFFE652F20EEE
:103B00000101FF17ABAC03D0FF91ABB0FF81ABB4A9
:103B1000FF85ABB2FF87AE50DF6EDF50E552E55256
:103B2000E5CFDAFFE7CFD9FF1200D9CFE6FFDACF32
:103B3000E6FFE1CFD9FFE2CFDAFFE652E652FC0E14
:103B4000DBCFDEFFDBCFDDFF010EDB50CF6EDF50C2
:103B5000CE6EE552E552E552E5CFDAFFE7CFD9FF69
:103B60001200D9CFE6FFDACFE6FFE1CFD9FFE2CFEF
:103B7000DAFF3F0EC716C66AC56AFD0EDB50C612D5
:103B8000FC0EDB50C712C68AE552E5CFDAFFE7CF5D
:103B9000D9FF1200FF0EE3502D6EEF0E01D0F30E91
:103BA000E76EE72ED1EF1DF00C0E2C6EE76AE72EC4
:103BB000D7EF1DF02C2ED6EF1DF02D2ECFEF1DF0E0
:103BC0001200D9CFE6FFDACFE6FFE1CFD9FFE2CF8F
:103BD000DAFFACAC04D0AC900101FFB3AC80FD0EB9
:103BE000DB50AD6EE552E5CFDAFFE7CFD9FF12002B
:103BF000F36AF46AFF0EE124E96EFF0EE220EA6E3A
:103C0000ED6607D02F0EEF6404D03A0EEF6001D0BE
:103C1000F32A1200380EF36E00EE00F00F0E01D8FA
:103C20001200EA6002D0EE6AFCD7F350E96012009D
:103C3000EE6AFCD71EEE00F02EEE00F0F86A279C2C
:103C40008FEC1BF05BEC1EF0E5EC0AF0FBD71200EA
:103C5000FF0EE350ACBA04D0AF6AAB8EAC8A949C32
:103C6000ACA2FED7AD6EF36EF46A1200FF0EE35005
:103C7000E84E1200000000D000D000D0E82EFAD7A5
:103C80001200C450036E026AC3500210F36E03C0E8
:103C9000F4FF12003031323334353637383961624F
:103CA0006364656600FFC250020B01E0010E120062
:103CB000C282120012001200802500008B35B1353F
:103CC000D135F9350A360E362C3641368B35B135BD
:103CD000D135F9350A360E362C3641363030303093
:103CE00030303030003132333435363738393031D6
:103CF000323334353600980A4A616E762E004665B6
:103D000076722E004D6172732000417672696C00EC
:103D10004D61692020004A75696E20004A75696C02
:103D20002E00416F75742000536570742E004F6330
:103D3000746F2E004E6F76652E00446563652E000D
:103D400044696D616E004C756E6469004D6172640A
:103D500069004D65726372004A6575646900566555
:103D60006E64720053616D656400FFFFFFFFFFFF2B
:103D7000FFFFFFFFFFFFFFFFFFFFFFFFFFFFFFFF53
:103D8000FFFFFFFFFFFFFFFFFFFFFFFFFFFFFFFF43
:103D9000FFFFFFFFFFFFFFFFFFFFFFFFFFFFFFFF33
:103DA000FFFFFFFFFFFFFFFFFFFFFFFFFFFFFFFF23
:0200000400F00A
:1000000050726F6A65743A31384632364B3232205C
:1000100020554152543120425420200D0000000050
:1000200056657273696F6E20323330562035304812
:100030007A2020202020202020202020200D0A00AF
:10004000506F727420436F6D206F757665727420E7
:100050002620496E69742048415244572E0D0A00EB
:10006000426F75636C6520656E2032205365632096
:1000700020203C4553433E2065786974200D0A00DA
:1000800041766563205541525431204841524457CE
:100090004152452E2E2E2E2E2E2E2E2E2E0D0A00A5
:1000A0007061756C666A756A6F40667265652E660A
:1000B0007220202020202020202020202020200D01
:1000C0004D504C4142204944452056382E3931206C
:1000D0002020202020202020202020202020200D33
:1000E0004331382076332E34352E303020202050C6
:1000F00069634B697433202020202020200D0A00E2
:10010000312E6D657373616765206F76657220317E
:100110003030682E2E2E2E2020202020230D0A0085
:10012000322E6D657373616765206F76657220315D
:100130003230682E2E2E2E20202020202A0D0A005C
:1001400020202020202020202020202020202020AF
:1001500020202020202020202020202020200000DF
:10016000FFFFFFFFFFFFFFFFFFFFFFFFFFFFFFFF9F
:10017000FFFFFFFFFFFFFFFFFFFFFFFFFFFFFFFF8F
:10018000FFFFFFFFFFFFFFFFFFFFFFFFFFFFFFFF7F
:10019000FFFFFFFFFFFFFFFFFFFFFFFFFFFFFFFF6F
:1001A000FFFFFFFFFFFFFFFFFFFFFFFFFFFFFFFF5F
:1001B000FFFFFFFFFFFFFFFFFFFFFFFFFFFFFFFF4F
:1001C000FFFFFFFFFFFFFFFFFFFFFFFFFFFFFFFF3F
:1001D000FFFFFFFFFFFFFFFFFFFFFFFFFFFFFFFF2F
:1001E000FFFFFFFFFFFFFFFFFFFFFFFFFFFFFFFF1F
:1001F000FFFFFFFFFFFFFFFFFFFFFFFFFFFFFFFF0F
:1002000020202020202020202020202020202020EE
:100210002020202031384632364B32325F5365631E
:10022000746575725F3530485254432D44533133F1
:100230003037202B204C434420493243566572739B
:100240007573203133303931372043313820202045
:10025000496E69742055415254312039363030622C
:1002600064732020496E69742052544320445331F2
:100270003330372020202020496E6974206D6F6450
:10028000756C652059432D4D435520204E6F206CD1
:10029000696E6B20696620617070616972656420A7
:1002A00031384632364B32325F42545F59435F4DEC
:1002B000435520206C696E6B656420746F2041701B
:1002C00070696E76656E742E2020202020202020FC
:1002D000202020202020202020202020FFFFFFFFA2
:1002E000FFFFFFFFFFFFFFFFFFFFFFFFFFFFFFFF1E
:1002F000FFFFFFFFFFFFFFFFFFFFFFFFFFFFFFFF0E
:10030000FFFFFFFFFFFFFFFFFFFFFFFFFFFFFFFFFD
:10031000FFFFFFFFFFFFFFFFFFFFFFFFFFFFFFFFED
:10032000FFFFFFFFFFFFFFFFFFFFFFFFFFFFFFFFDD
:10033000FFFFFFFFFFFFFFFFFFFFFFFFFFFFFFFFCD
:10034000FFFFFFFFFFFFFFFFFFFFFFFFFFFFFFFFBD
:10035000FFFFFFFFFFFFFFFFFFFFFFFFFFFFFFFFAD
:10036000FFFFFFFFFFFFFFFFFFFFFFFFFFFFFFFF9D
:10037000FFFFFFFFFFFFFFFFFFFFFFFFFFFFFFFF8D
:10038000FFFFFFFFFFFFFFFFFFFFFFFFFFFFFFFF7D
:10039000FFFFFFFFFFFFFFFFFFFFFFFFFFFFFFFF6D
:1003A000FFFFFFFFFFFFFFFFFFFFFFFFFFFFFFFF5D
:1003B000FFFFFFFFFFFFFFFFFFFFFFFFFFFFFFFF4D
:1003C000FFFFFFFFFFFFFFFFFFFFFFFFFFFFFFFF3D
:1003D000FFFFFFFFFFFFFFFFFFFFFFFFFFFFFFFF2D
:1003E000FFFFFFFFFFFFFFFFFFFFFFFFFFFFFFFF1D
:1003F000FFFFFFFFFFFFFFFFFFFFFFFFFFFFFFFF0D
:020000040030CA
:0E0000000023193C009D84000FC00FE00F404C
:020000040020DA
:08000000FFFFFFFFFFFFFFFF00
:00000001FF
